###############################################################################
#
# IAR ELF Linker V7.20.5.7591/W32 for ARM                 14/Oct/2014  17:19:17
# Copyright 2007-2014 IAR Systems AB.
#
#    Output file  =  
#        C:\ESEMPI-SW\STM32L0\STM32Cube_FW_L0_V1.1.0\Projects\STM32L053C8-Discovery\Demonstrations\EWARM\STM32L0538-Discovery\Exe\Project.out
#    Map file     =  
#        C:\ESEMPI-SW\STM32L0\STM32Cube_FW_L0_V1.1.0\Projects\STM32L053C8-Discovery\Demonstrations\EWARM\STM32L0538-Discovery\List\Project.map
#    Command line =  
#        C:\ESEMPI-SW\STM32L0\STM32Cube_FW_L0_V1.1.0\Projects\STM32L053C8-Discovery\Demonstrations\EWARM\STM32L0538-Discovery\Obj\bsp.o
#        C:\ESEMPI-SW\STM32L0\STM32Cube_FW_L0_V1.1.0\Projects\STM32L053C8-Discovery\Demonstrations\EWARM\STM32L0538-Discovery\Obj\gde021a1.o
#        C:\ESEMPI-SW\STM32L0\STM32Cube_FW_L0_V1.1.0\Projects\STM32L053C8-Discovery\Demonstrations\EWARM\STM32L0538-Discovery\Obj\main.o
#        C:\ESEMPI-SW\STM32L0\STM32Cube_FW_L0_V1.1.0\Projects\STM32L053C8-Discovery\Demonstrations\EWARM\STM32L0538-Discovery\Obj\menu.o
#        C:\ESEMPI-SW\STM32L0\STM32Cube_FW_L0_V1.1.0\Projects\STM32L053C8-Discovery\Demonstrations\EWARM\STM32L0538-Discovery\Obj\power.o
#        C:\ESEMPI-SW\STM32L0\STM32Cube_FW_L0_V1.1.0\Projects\STM32L053C8-Discovery\Demonstrations\EWARM\STM32L0538-Discovery\Obj\startup_stm32l053xx.o
#        C:\ESEMPI-SW\STM32L0\STM32Cube_FW_L0_V1.1.0\Projects\STM32L053C8-Discovery\Demonstrations\EWARM\STM32L0538-Discovery\Obj\stm32l0538_discovery.o
#        C:\ESEMPI-SW\STM32L0\STM32Cube_FW_L0_V1.1.0\Projects\STM32L053C8-Discovery\Demonstrations\EWARM\STM32L0538-Discovery\Obj\stm32l0538_discovery_epd.o
#        C:\ESEMPI-SW\STM32L0\STM32Cube_FW_L0_V1.1.0\Projects\STM32L053C8-Discovery\Demonstrations\EWARM\STM32L0538-Discovery\Obj\stm32l0xx_hal.o
#        C:\ESEMPI-SW\STM32L0\STM32Cube_FW_L0_V1.1.0\Projects\STM32L053C8-Discovery\Demonstrations\EWARM\STM32L0538-Discovery\Obj\stm32l0xx_hal_cortex.o
#        C:\ESEMPI-SW\STM32L0\STM32Cube_FW_L0_V1.1.0\Projects\STM32L053C8-Discovery\Demonstrations\EWARM\STM32L0538-Discovery\Obj\stm32l0xx_hal_dma.o
#        C:\ESEMPI-SW\STM32L0\STM32Cube_FW_L0_V1.1.0\Projects\STM32L053C8-Discovery\Demonstrations\EWARM\STM32L0538-Discovery\Obj\stm32l0xx_hal_flash.o
#        C:\ESEMPI-SW\STM32L0\STM32Cube_FW_L0_V1.1.0\Projects\STM32L053C8-Discovery\Demonstrations\EWARM\STM32L0538-Discovery\Obj\stm32l0xx_hal_flash_ex.o
#        C:\ESEMPI-SW\STM32L0\STM32Cube_FW_L0_V1.1.0\Projects\STM32L053C8-Discovery\Demonstrations\EWARM\STM32L0538-Discovery\Obj\stm32l0xx_hal_gpio.o
#        C:\ESEMPI-SW\STM32L0\STM32Cube_FW_L0_V1.1.0\Projects\STM32L053C8-Discovery\Demonstrations\EWARM\STM32L0538-Discovery\Obj\stm32l0xx_hal_i2c.o
#        C:\ESEMPI-SW\STM32L0\STM32Cube_FW_L0_V1.1.0\Projects\STM32L053C8-Discovery\Demonstrations\EWARM\STM32L0538-Discovery\Obj\stm32l0xx_hal_i2c_ex.o
#        C:\ESEMPI-SW\STM32L0\STM32Cube_FW_L0_V1.1.0\Projects\STM32L053C8-Discovery\Demonstrations\EWARM\STM32L0538-Discovery\Obj\stm32l0xx_hal_msp.o
#        C:\ESEMPI-SW\STM32L0\STM32Cube_FW_L0_V1.1.0\Projects\STM32L053C8-Discovery\Demonstrations\EWARM\STM32L0538-Discovery\Obj\stm32l0xx_hal_pcd.o
#        C:\ESEMPI-SW\STM32L0\STM32Cube_FW_L0_V1.1.0\Projects\STM32L053C8-Discovery\Demonstrations\EWARM\STM32L0538-Discovery\Obj\stm32l0xx_hal_pcd_ex.o
#        C:\ESEMPI-SW\STM32L0\STM32Cube_FW_L0_V1.1.0\Projects\STM32L053C8-Discovery\Demonstrations\EWARM\STM32L0538-Discovery\Obj\stm32l0xx_hal_pwr.o
#        C:\ESEMPI-SW\STM32L0\STM32Cube_FW_L0_V1.1.0\Projects\STM32L053C8-Discovery\Demonstrations\EWARM\STM32L0538-Discovery\Obj\stm32l0xx_hal_pwr_ex.o
#        C:\ESEMPI-SW\STM32L0\STM32Cube_FW_L0_V1.1.0\Projects\STM32L053C8-Discovery\Demonstrations\EWARM\STM32L0538-Discovery\Obj\stm32l0xx_hal_rcc.o
#        C:\ESEMPI-SW\STM32L0\STM32Cube_FW_L0_V1.1.0\Projects\STM32L053C8-Discovery\Demonstrations\EWARM\STM32L0538-Discovery\Obj\stm32l0xx_hal_rcc_ex.o
#        C:\ESEMPI-SW\STM32L0\STM32Cube_FW_L0_V1.1.0\Projects\STM32L053C8-Discovery\Demonstrations\EWARM\STM32L0538-Discovery\Obj\stm32l0xx_hal_spi.o
#        C:\ESEMPI-SW\STM32L0\STM32Cube_FW_L0_V1.1.0\Projects\STM32L053C8-Discovery\Demonstrations\EWARM\STM32L0538-Discovery\Obj\stm32l0xx_hal_tsc.o
#        C:\ESEMPI-SW\STM32L0\STM32Cube_FW_L0_V1.1.0\Projects\STM32L053C8-Discovery\Demonstrations\EWARM\STM32L0538-Discovery\Obj\stm32l0xx_it.o
#        C:\ESEMPI-SW\STM32L0\STM32Cube_FW_L0_V1.1.0\Projects\STM32L053C8-Discovery\Demonstrations\EWARM\STM32L0538-Discovery\Obj\system_stm32l0xx.o
#        C:\ESEMPI-SW\STM32L0\STM32Cube_FW_L0_V1.1.0\Projects\STM32L053C8-Discovery\Demonstrations\EWARM\STM32L0538-Discovery\Obj\tsl.o
#        C:\ESEMPI-SW\STM32L0\STM32Cube_FW_L0_V1.1.0\Projects\STM32L053C8-Discovery\Demonstrations\EWARM\STM32L0538-Discovery\Obj\tsl_acq.o
#        C:\ESEMPI-SW\STM32L0\STM32Cube_FW_L0_V1.1.0\Projects\STM32L053C8-Discovery\Demonstrations\EWARM\STM32L0538-Discovery\Obj\tsl_acq_tsc.o
#        C:\ESEMPI-SW\STM32L0\STM32Cube_FW_L0_V1.1.0\Projects\STM32L053C8-Discovery\Demonstrations\EWARM\STM32L0538-Discovery\Obj\tsl_dxs.o
#        C:\ESEMPI-SW\STM32L0\STM32Cube_FW_L0_V1.1.0\Projects\STM32L053C8-Discovery\Demonstrations\EWARM\STM32L0538-Discovery\Obj\tsl_ecs.o
#        C:\ESEMPI-SW\STM32L0\STM32Cube_FW_L0_V1.1.0\Projects\STM32L053C8-Discovery\Demonstrations\EWARM\STM32L0538-Discovery\Obj\tsl_filter.o
#        C:\ESEMPI-SW\STM32L0\STM32Cube_FW_L0_V1.1.0\Projects\STM32L053C8-Discovery\Demonstrations\EWARM\STM32L0538-Discovery\Obj\tsl_globals.o
#        C:\ESEMPI-SW\STM32L0\STM32Cube_FW_L0_V1.1.0\Projects\STM32L053C8-Discovery\Demonstrations\EWARM\STM32L0538-Discovery\Obj\tsl_linrot.o
#        C:\ESEMPI-SW\STM32L0\STM32Cube_FW_L0_V1.1.0\Projects\STM32L053C8-Discovery\Demonstrations\EWARM\STM32L0538-Discovery\Obj\tsl_object.o
#        C:\ESEMPI-SW\STM32L0\STM32Cube_FW_L0_V1.1.0\Projects\STM32L053C8-Discovery\Demonstrations\EWARM\STM32L0538-Discovery\Obj\tsl_time.o
#        C:\ESEMPI-SW\STM32L0\STM32Cube_FW_L0_V1.1.0\Projects\STM32L053C8-Discovery\Demonstrations\EWARM\STM32L0538-Discovery\Obj\tsl_touchkey.o
#        C:\ESEMPI-SW\STM32L0\STM32Cube_FW_L0_V1.1.0\Projects\STM32L053C8-Discovery\Demonstrations\EWARM\STM32L0538-Discovery\Obj\tsl_user.o
#        C:\ESEMPI-SW\STM32L0\STM32Cube_FW_L0_V1.1.0\Projects\STM32L053C8-Discovery\Demonstrations\EWARM\STM32L0538-Discovery\Obj\usbd_conf.o
#        C:\ESEMPI-SW\STM32L0\STM32Cube_FW_L0_V1.1.0\Projects\STM32L053C8-Discovery\Demonstrations\EWARM\STM32L0538-Discovery\Obj\usbd_core.o
#        C:\ESEMPI-SW\STM32L0\STM32Cube_FW_L0_V1.1.0\Projects\STM32L053C8-Discovery\Demonstrations\EWARM\STM32L0538-Discovery\Obj\usbd_ctlreq.o
#        C:\ESEMPI-SW\STM32L0\STM32Cube_FW_L0_V1.1.0\Projects\STM32L053C8-Discovery\Demonstrations\EWARM\STM32L0538-Discovery\Obj\usbd_desc.o
#        C:\ESEMPI-SW\STM32L0\STM32Cube_FW_L0_V1.1.0\Projects\STM32L053C8-Discovery\Demonstrations\EWARM\STM32L0538-Discovery\Obj\usbd_hid.o
#        C:\ESEMPI-SW\STM32L0\STM32Cube_FW_L0_V1.1.0\Projects\STM32L053C8-Discovery\Demonstrations\EWARM\STM32L0538-Discovery\Obj\usbd_ioreq.o
#        C:\ESEMPI-SW\STM32L0\STM32Cube_FW_L0_V1.1.0\Projects\STM32L053C8-Discovery\Demonstrations\EWARM\STM32L0538-Discovery\Obj\usbdapp.o
#        -o
#        C:\ESEMPI-SW\STM32L0\STM32Cube_FW_L0_V1.1.0\Projects\STM32L053C8-Discovery\Demonstrations\EWARM\STM32L0538-Discovery\Exe\Project.out
#        --map
#        C:\ESEMPI-SW\STM32L0\STM32Cube_FW_L0_V1.1.0\Projects\STM32L053C8-Discovery\Demonstrations\EWARM\STM32L0538-Discovery\List\Project.map
#        --config
#        C:\ESEMPI-SW\STM32L0\STM32Cube_FW_L0_V1.1.0\Projects\STM32L053C8-Discovery\Demonstrations\EWARM\stm32l053xx_flash.icf
#        --entry __iar_program_start --vfe
#
###############################################################################

*******************************************************************************
*** RUNTIME MODEL ATTRIBUTES
***

CppFlavor       = *
__SystemLibrary = DLib


*******************************************************************************
*** PLACEMENT SUMMARY
***

"A1":  place at 0x08000000 { ro section .intvec };
"P1":  place in [from 0x08000000 to 0x0800ffff] { ro };
"P2":  place in [from 0x20000000 to 0x20001fff] { rw, block CSTACK, block HEAP };

  Section            Kind        Address    Size  Object
  -------            ----        -------    ----  ------
"A1":                                       0xc0
  .intvec            ro code  0x08000000    0xc0  startup_stm32l053xx.o [1]
                            - 0x080000c0    0xc0

"P1":                                     0x8373
  .rodata            const    0x080000c0  0x1bd8  stm32l0538_discovery_epd.o [1]
  .text              ro code  0x08001c98   0xcc4  stm32l0xx_hal_pcd.o [1]
  .text              ro code  0x0800295c   0x226  usbd_conf.o [1]
  .text              ro code  0x08002b82    0x2a  zero_init3.o [4]
  .text              ro code  0x08002bac   0x27c  stm32l0xx_hal_gpio.o [1]
  .text              ro code  0x08002e28    0x94  stm32l0xx_hal_cortex.o [1]
  .text              ro code  0x08002ebc   0x26c  usbd_core.o [1]
  .text              ro code  0x08003128    0x36  stm32l0xx_hal_pcd_ex.o [1]
  .text              ro code  0x0800315e     0xa  xsprout.o [3]
  .text              ro code  0x08003168   0x7a0  menu.o [1]
  .text              ro code  0x08003908   0x3d0  usbd_ctlreq.o [1]
  .text              ro code  0x08003cd8    0x60  usbd_ioreq.o [1]
  .text              ro code  0x08003d38    0xe0  I32DivModFast.o [4]
  .text              ro code  0x08003e18   0x268  stm32l0538_discovery_epd.o [1]
  .text              ro code  0x08004080    0x98  stm32l0xx_hal.o [1]
  .text              ro code  0x08004118    0xb4  tsl_user.o [1]
  .text              ro code  0x080041cc    0x98  bsp.o [1]
  .text              ro code  0x08004264    0x70  usbdapp.o [1]
  .text              ro code  0x080042d4   0x2b5  stm32l0538_discovery.o [1]
  .text              ro code  0x0800458a     0x2  startup_stm32l053xx.o [1]
  .text              ro code  0x0800458c   0x6e4  power.o [1]
  .text              ro code  0x08004c70    0xdc  stm32l0xx_hal_tsc.o [1]
  .text              ro code  0x08004d4c   0x66c  stm32l0xx_hal_rcc.o [1]
  .text              ro code  0x080053b8   0x1d4  stm32l0xx_hal_rcc_ex.o [1]
  .text              ro code  0x0800558c     0x2  IntDivZer.o [4]
  .text              ro code  0x0800558e     0x2  startup_stm32l053xx.o [1]
  .text              ro code  0x08005590   0x170  stm32l0xx_hal_msp.o [1]
  .text              ro code  0x08005700    0xc0  tsl_object.o [1]
  .text              ro code  0x080057c0    0x30  tsl.o [1]
  .text              ro code  0x080057f0    0xe8  tsl_acq_tsc.o [1]
  .text              ro code  0x080058d8   0x14c  tsl_acq.o [1]
  .text              ro code  0x08005a24     0x2  tsl_dxs.o [1]
  .text              ro code  0x08005a26     0x2  startup_stm32l053xx.o [1]
  .text              ro code  0x08005a28    0x86  tsl_time.o [1]
  .text              ro code  0x08005aae     0x2  startup_stm32l053xx.o [1]
  .text              ro code  0x08005ab0   0x1f0  tsl_ecs.o [1]
  .text              ro code  0x08005ca0   0x140  usbd_hid.o [1]
  .text              ro code  0x08005de0   0x2dc  stm32l0xx_hal_spi.o [1]
  .text              ro code  0x080060bc   0x5c0  stm32l0xx_hal_i2c.o [1]
  .text              ro code  0x0800667c    0x38  sprintf.o [3]
  .text              ro code  0x080066b4    0x30  stm32l0xx_hal_pwr.o [1]
  .text              ro code  0x080066e4    0x1c  stm32l0xx_hal_pwr_ex.o [1]
  .text              ro code  0x08006700   0x524  xprintfsmall_nomb.o [3]
  .text              ro code  0x08006c24    0x14  strchr.o [4]
  .text              ro code  0x08006c38    0x10  strlen.o [4]
  .text              ro code  0x08006c48    0x18  memchr.o [4]
  .text              ro code  0x08006c60   0xc08  tsl_linrot.o [1]
  .text              ro code  0x08007868   0x2d8  gde021a1.o [1]
  .text              ro code  0x08007b40   0x1be  lz77_init.o [4]
  .text              ro code  0x08007cfe     0xa  abort.o [3]
  .text              ro code  0x08007d08     0xc  XXexit.o [4]
  .rodata            const    0x08007d14   0x10c  tsl_user.o [1]
  .text              ro code  0x08007e20   0x108  usbd_desc.o [1]
  .text              ro code  0x08007f28    0x62  stm32l0xx_it.o [1]
  .text              ro code  0x08007f8a     0x2  startup_stm32l053xx.o [1]
  .text              ro code  0x08007f8c    0x58  system_stm32l0xx.o [1]
  .rodata            const    0x08007fe4    0x50  menu.o [1]
  .text              ro code  0x08008034    0x28  data_init.o [4]
  .iar.init_table    const    0x0800805c    0x2c  - Linker created -
  .text              ro code  0x08008088    0x1a  cmain.o [4]
  .text              ro code  0x080080a2     0x4  low_level_init.o [3]
  .text              ro code  0x080080a6    0x14  main.o [1]
  .text              ro code  0x080080ba     0x8  exit.o [3]
  .text              ro code  0x080080c2     0x2  startup_stm32l053xx.o [1]
  .text              ro code  0x080080c4     0xa  cexit.o [4]
  .text              ro code  0x080080ce     0x2  startup_stm32l053xx.o [1]
  .rodata            const    0x080080d0    0x14  tsl_linrot.o [1]
  .text              ro code  0x080080e4    0x10  startup_stm32l053xx.o [1]
  .text              ro code  0x080080f4     0xc  cstartup_M.o [4]
  .text              ro code  0x08008100     0x2  startup_stm32l053xx.o [1]
  .text              ro code  0x08008102     0x2  startup_stm32l053xx.o [1]
  .text              ro code  0x08008104     0x2  startup_stm32l053xx.o [1]
  .text              ro code  0x08008106     0x2  startup_stm32l053xx.o [1]
  .text              ro code  0x08008108     0x2  startup_stm32l053xx.o [1]
  .text              ro code  0x0800810a     0x2  startup_stm32l053xx.o [1]
  .text              ro code  0x0800810c     0x2  startup_stm32l053xx.o [1]
  .text              ro code  0x0800810e     0x2  startup_stm32l053xx.o [1]
  .text              ro code  0x08008110     0x2  startup_stm32l053xx.o [1]
  .text              ro code  0x08008112     0x2  startup_stm32l053xx.o [1]
  .text              ro code  0x08008114     0x2  startup_stm32l053xx.o [1]
  .text              ro code  0x08008116     0x2  startup_stm32l053xx.o [1]
  .text              ro code  0x08008118     0x2  startup_stm32l053xx.o [1]
  .text              ro code  0x0800811a     0x2  startup_stm32l053xx.o [1]
  .text              ro code  0x0800811c     0x2  startup_stm32l053xx.o [1]
  .text              ro code  0x0800811e     0x2  startup_stm32l053xx.o [1]
  .text              ro code  0x08008120     0x2  startup_stm32l053xx.o [1]
  .rodata            const    0x08008122     0x0  zero_init3.o [4]
  .rodata            const    0x08008122     0x0  lz77_init.o [4]
  Initializer bytes  ro data  0x08008122   0x311  <for P2 s0>
                            - 0x08008433  0x8373

"P2":                                     0x1898
  P2 s0                       0x20000000   0xa08  <Init block>
    .data            inited   0x20000000   0x85c  menu.o [1]
    .data            inited   0x2000085c    0x58  usbd_hid.o [1]
    .data            inited   0x200008b4    0x38  usbd_hid.o [1]
    .data            inited   0x200008ec    0x24  usbd_hid.o [1]
    .data            inited   0x20000910    0x20  gde021a1.o [1]
    .data            inited   0x20000930    0x20  system_stm32l0xx.o [1]
    .data            inited   0x20000950    0x1c  tsl_user.o [1]
    .data            inited   0x2000096c    0x1c  usbd_desc.o [1]
    .data            inited   0x20000988    0x1c  usbd_desc.o [1]
    .data            inited   0x200009a4    0x18  stm32l0538_discovery_epd.o [1]
    .data            inited   0x200009bc    0x10  stm32l0xx_hal_rcc.o [1]
    .data            inited   0x200009cc    0x10  tsl_user.o [1]
    .data            inited   0x200009dc     0xc  stm32l0xx_hal_rcc.o [1]
    .data            inited   0x200009e8     0xc  usbd_hid.o [1]
    .data            inited   0x200009f4     0x8  stm32l0538_discovery.o [1]
    .data            inited   0x200009fc     0x8  stm32l0538_discovery_epd.o [1]
    .data            inited   0x20000a04     0x4  stm32l0538_discovery.o [1]
  .bss               zero     0x20000a08   0x224  bsp.o [1]
  .bss               zero     0x20000c2c   0x178  usbd_conf.o [1]
  .bss               zero     0x20000da4   0x100  usbd_desc.o [1]
  .bss               zero     0x20000ea4    0x6c  power.o [1]
  .bss               zero     0x20000f10    0x64  menu.o [1]
  .bss               zero     0x20000f74    0x54  stm32l0538_discovery.o [1]
  .bss               zero     0x20000fc8    0x40  bsp.o [1]
  .bss               zero     0x20001008    0x24  tsl_user.o [1]
  .bss               zero     0x2000102c    0x18  menu.o [1]
  .bss               zero     0x20001044    0x18  tsl_globals.o [1]
  .bss               zero     0x2000105c    0x10  tsl_user.o [1]
  .bss               zero     0x2000106c    0x10  usbd_conf.o [1]
  .bss               zero     0x2000107c     0x8  tsl_user.o [1]
  .bss               zero     0x20001084     0x4  stm32l0xx_hal.o [1]
  .bss               zero     0x20001088     0x4  stm32l0xx_it.o [1]
  .bss               zero     0x2000108c     0x4  usbdapp.o [1]
  .bss               zero     0x20001090     0x2  tsl_linrot.o [1]
  .bss               zero     0x20001092     0x1  usbd_ctlreq.o [1]
  CSTACK                      0x20001098   0x800  <Block>
    CSTACK           uninit   0x20001098   0x800  <Block tail>
                            - 0x20001898  0x1898


*******************************************************************************
*** INIT TABLE
***

          Address     Size
          -------     ----
Zero (__iar_zero_init3)
    1 destination range, total size 0x68b:
          0x20000a08  0x68b

Copy/lz77 (__iar_lz77_init3)
    1 source range, total size 0x311 (30% of destination):
          0x08008122  0x311
    1 destination range, total size 0xa08:
          0x20000000  0xa08



*******************************************************************************
*** MODULE SUMMARY
***

    Module                      ro code  ro data  rw data
    ------                      -------  -------  -------
C:\ESEMPI-SW\STM32L0\STM32Cube_FW_L0_V1.1.0\Projects\STM32L053C8-Discovery\Demonstrations\EWARM\STM32L0538-Discovery\Obj: [1]
    bsp.o                           152               612
    gde021a1.o                      728        9       32
    main.o                           20
    menu.o                        1 952      734    2 264
    power.o                       1 764               108
    startup_stm32l053xx.o           256
    stm32l0538_discovery.o          693        5       96
    stm32l0538_discovery_epd.o      616    7 137       32
    stm32l0xx_hal.o                 152                 4
    stm32l0xx_hal_cortex.o          148
    stm32l0xx_hal_gpio.o            636
    stm32l0xx_hal_i2c.o           1 472
    stm32l0xx_hal_msp.o             368
    stm32l0xx_hal_pcd.o           3 268
    stm32l0xx_hal_pcd_ex.o           54
    stm32l0xx_hal_pwr.o              48
    stm32l0xx_hal_pwr_ex.o           28
    stm32l0xx_hal_rcc.o           1 644        9       28
    stm32l0xx_hal_rcc_ex.o          468
    stm32l0xx_hal_spi.o             732
    stm32l0xx_hal_tsc.o             220
    stm32l0xx_it.o                   98                 4
    system_stm32l0xx.o               88       10       32
    tsl.o                            48
    tsl_acq.o                       332
    tsl_acq_tsc.o                   232
    tsl_dxs.o                         2
    tsl_ecs.o                       496
    tsl_globals.o                                      24
    tsl_linrot.o                  3 080       20        2
    tsl_object.o                    192
    tsl_time.o                      134
    tsl_user.o                      180      282      104
    usbd_conf.o                     550               392
    usbd_core.o                     620
    usbd_ctlreq.o                   976                 1
    usbd_desc.o                     264       17      312
    usbd_hid.o                      320       58      192
    usbd_ioreq.o                     96
    usbdapp.o                       112                 4
    -----------------------------------------------------
    Total:                       23 239    8 281    4 243

command line: [2]
    -----------------------------------------------------
    Total:

dl6M_tlf.a: [3]
    abort.o                          10
    exit.o                            8
    low_level_init.o                  4
    sprintf.o                        56
    xprintfsmall_nomb.o           1 316
    xsprout.o                        10
    -----------------------------------------------------
    Total:                        1 404

rt6M_tl.a: [4]
    I32DivModFast.o                 224
    IntDivZer.o                       2
    XXexit.o                         12
    cexit.o                          10
    cmain.o                          26
    cstartup_M.o                     12
    data_init.o                      40
    lz77_init.o                     446
    memchr.o                         24
    strchr.o                         20
    strlen.o                         16
    zero_init3.o                     42
    -----------------------------------------------------
    Total:                          874

    Gaps                              1
    Linker created                            44    2 048
---------------------------------------------------------
    Grand Total:                 25 518    8 325    6 291


*******************************************************************************
*** ENTRY LIST
***

Entry                      Address    Size  Type      Object
-----                      -------    ----  ----      ------
?main                   0x08008089          Code  Gb  cmain.o [4]
AHBPrescTable           0x20000930    0x10  Data  Gb  system_stm32l0xx.o [1]
APBAHBPrescTable        0x200009bc    0x10  Data  Lc  stm32l0xx_hal_rcc.o [1]
BSP_EPD_Clear           0x08003e59    0x24  Code  Gb  stm32l0538_discovery_epd.o [1]
BSP_EPD_DisplayChar     0x08003e7d    0x4c  Code  Gb  stm32l0538_discovery_epd.o [1]
BSP_EPD_DisplayStringAt
                        0x08003ec9    0x98  Code  Gb  stm32l0538_discovery_epd.o [1]
BSP_EPD_DrawHLine       0x08003f61    0x26  Code  Gb  stm32l0538_discovery_epd.o [1]
BSP_EPD_DrawImage       0x08003fe1    0x5e  Code  Gb  stm32l0538_discovery_epd.o [1]
BSP_EPD_DrawRect        0x08003fad    0x34  Code  Gb  stm32l0538_discovery_epd.o [1]
BSP_EPD_DrawVLine       0x08003f87    0x26  Code  Gb  stm32l0538_discovery_epd.o [1]
BSP_EPD_GetXSize        0x08003e3b     0xc  Code  Gb  stm32l0538_discovery_epd.o [1]
BSP_EPD_GetYSize        0x08003e47     0xc  Code  Gb  stm32l0538_discovery_epd.o [1]
BSP_EPD_Init            0x08003e19    0x22  Code  Gb  stm32l0538_discovery_epd.o [1]
BSP_EPD_RefreshDisplay  0x0800403f    0x2c  Code  Gb  stm32l0538_discovery_epd.o [1]
BSP_EPD_SetFont         0x08003e53     0x6  Code  Gb  stm32l0538_discovery_epd.o [1]
BSP_LED_Init            0x080042d5    0x42  Code  Gb  stm32l0538_discovery.o [1]
BSP_LED_Off             0x08004319     0x4  Code  Gb  stm32l0538_discovery.o [1]
BSP_LED_Toggle          0x08004331    0x16  Code  Gb  stm32l0538_discovery.o [1]
BSP_PB_Init             0x08004349    0x6c  Code  Gb  stm32l0538_discovery.o [1]
BSP_TSL_Init            0x080041ed    0x44  Code  Gb  bsp.o [1]
BSP_USB_Init            0x08004231    0x1e  Code  Gb  bsp.o [1]
BUTTON_IRQn             0x08004588     0x1  Data  Gb  stm32l0538_discovery.o [1]
BUTTON_PIN              0x08004584     0x2  Data  Gb  stm32l0538_discovery.o [1]
BUTTON_PORT             0x20000a04     0x4  Data  Gb  stm32l0538_discovery.o [1]
Background_pic          0x20000008   0x60c  Data  Lc  menu.o [1]
Bsp_Init                0x080041cd    0x20  Code  Gb  bsp.o [1]
ButtonPressed           0x20000004     0x4  Data  Gb  menu.o [1]
CSTACK$$Base            0x20001098           --   Gb  - Linker created -
CSTACK$$Limit           0x20001898           --   Gb  - Linker created -
CalibDiv                0x20001090     0x2  Data  Lc  tsl_linrot.o [1]
DebugMon_Handler        0x08007f2f     0x2  Code  Gb  stm32l0xx_it.o [1]
ECSLastTick             0x20000958     0x2  Data  Gb  tsl_user.o [1]
EPD_Delay               0x08004579     0x8  Code  Gb  stm32l0538_discovery.o [1]
EPD_IO_Init             0x08004457    0xae  Code  Gb  stm32l0538_discovery.o [1]
EPD_IO_WriteData        0x08004505    0x24  Code  Gb  stm32l0538_discovery.o [1]
EPD_IO_WriteReg         0x08004529    0x22  Code  Gb  stm32l0538_discovery.o [1]
EXTI0_1_IRQHandler      0x08007f75     0xa  Code  Gb  stm32l0xx_it.o [1]
EXTI4_15_IRQHandler     0x08007f7f     0xc  Code  Gb  stm32l0xx_it.o [1]
Font12                  0x200009b4     0x8  Data  Gb  stm32l0538_discovery_epd.o [1]
Font12_Table            0x08001114   0x7cc  Data  Gb  stm32l0538_discovery_epd.o [1]
Font16                  0x200009ac     0x8  Data  Gb  stm32l0538_discovery_epd.o [1]
Font16_Table            0x080000c0  0x1054  Data  Gb  stm32l0538_discovery_epd.o [1]
Font8                   0x200009fc     0x8  Data  Gb  stm32l0538_discovery_epd.o [1]
Font8_Table             0x080018e0   0x3b8  Data  Gb  stm32l0538_discovery_epd.o [1]
FullSlider_pic          0x20000614   0x248  Data  Lc  menu.o [1]
GPIOA_AFRH              0x20000f20     0x4  Data  Gb  menu.o [1]
GPIOA_AFRL              0x20000f1c     0x4  Data  Gb  menu.o [1]
GPIOA_MODER             0x20000f10     0x4  Data  Gb  menu.o [1]
GPIOA_OSPEEDR           0x20000f18     0x4  Data  Gb  menu.o [1]
GPIOA_OTYPER            0x20000f14     0x4  Data  Gb  menu.o [1]
GPIOB_AFRH              0x20000f34     0x4  Data  Gb  menu.o [1]
GPIOB_AFRL              0x20000f30     0x4  Data  Gb  menu.o [1]
GPIOB_MODER             0x20000f24     0x4  Data  Gb  menu.o [1]
GPIOB_OSPEEDR           0x20000f2c     0x4  Data  Gb  menu.o [1]
GPIOB_OTYPER            0x20000f28     0x4  Data  Gb  menu.o [1]
GPIOC_AFRH              0x20000f48     0x4  Data  Gb  menu.o [1]
GPIOC_AFRL              0x20000f44     0x4  Data  Gb  menu.o [1]
GPIOC_MODER             0x20000f38     0x4  Data  Gb  menu.o [1]
GPIOC_OSPEEDR           0x20000f40     0x4  Data  Gb  menu.o [1]
GPIOC_OTYPER            0x20000f3c     0x4  Data  Gb  menu.o [1]
GPIOD_AFRH              0x20000f5c     0x4  Data  Gb  menu.o [1]
GPIOD_AFRL              0x20000f58     0x4  Data  Gb  menu.o [1]
GPIOD_MODER             0x20000f4c     0x4  Data  Gb  menu.o [1]
GPIOD_OSPEEDR           0x20000f54     0x4  Data  Gb  menu.o [1]
GPIOD_OTYPER            0x20000f50     0x4  Data  Gb  menu.o [1]
GPIOH_AFRH              0x20000f70     0x4  Data  Gb  menu.o [1]
GPIOH_AFRL              0x20000f6c     0x4  Data  Gb  menu.o [1]
GPIOH_MODER             0x20000f60     0x4  Data  Gb  menu.o [1]
GPIOH_OSPEEDR           0x20000f68     0x4  Data  Gb  menu.o [1]
GPIOH_OTYPER            0x20000f64     0x4  Data  Gb  menu.o [1]
GPIO_PIN                0x08004580     0x4  Data  Gb  stm32l0538_discovery.o [1]
GPIO_PORT               0x200009f4     0x8  Data  Gb  stm32l0538_discovery.o [1]
GetPointerData          0x08004265    0x32  Code  Gb  usbdapp.o [1]
HAL_Delay               0x080040d7    0x18  Code  Wk  stm32l0xx_hal.o [1]
HAL_GPIO_DeInit         0x08002d39    0x9c  Code  Gb  stm32l0xx_hal_gpio.o [1]
HAL_GPIO_EXTI_Callback  0x080038b1     0xa  Code  Gb  menu.o [1]
HAL_GPIO_EXTI_IRQHandler
                        0x08002df5    0x14  Code  Gb  stm32l0xx_hal_gpio.o [1]
HAL_GPIO_Init           0x08002bad   0x18c  Code  Gb  stm32l0xx_hal_gpio.o [1]
HAL_GPIO_ReadPin        0x08002dd5     0xc  Code  Gb  stm32l0xx_hal_gpio.o [1]
HAL_GPIO_TogglePin      0x08002ded     0x8  Code  Gb  stm32l0xx_hal_gpio.o [1]
HAL_GPIO_WritePin       0x08002de1     0xc  Code  Gb  stm32l0xx_hal_gpio.o [1]
HAL_GetTick             0x080040d1     0x6  Code  Wk  stm32l0xx_hal.o [1]
HAL_I2C_DeInit          0x0800615b    0x30  Code  Gb  stm32l0xx_hal_i2c.o [1]
HAL_I2C_Init            0x080060bd    0x9e  Code  Gb  stm32l0xx_hal_i2c.o [1]
HAL_I2C_Mem_Read        0x080062ad   0x11c  Code  Gb  stm32l0xx_hal_i2c.o [1]
HAL_I2C_Mem_Write       0x08006199   0x114  Code  Gb  stm32l0xx_hal_i2c.o [1]
HAL_I2C_MspDeInit       0x080056b3    0x32  Code  Gb  stm32l0xx_hal_msp.o [1]
HAL_I2C_MspInit         0x08005659    0x5a  Code  Gb  stm32l0xx_hal_msp.o [1]
HAL_IncTick             0x080040c7     0xa  Code  Wk  stm32l0xx_hal.o [1]
HAL_Init                0x08004081    0x22  Code  Gb  stm32l0xx_hal.o [1]
HAL_InitTick            0x080040a3    0x24  Code  Wk  stm32l0xx_hal.o [1]
HAL_MspInit             0x08005591     0x2  Code  Gb  stm32l0xx_hal_msp.o [1]
HAL_NVIC_DisableIRQ     0x08002e71     0xe  Code  Gb  stm32l0xx_hal_cortex.o [1]
HAL_NVIC_EnableIRQ      0x08002e63     0xe  Code  Gb  stm32l0xx_hal_cortex.o [1]
HAL_NVIC_SetPriority    0x08002e5b     0x8  Code  Gb  stm32l0xx_hal_cortex.o [1]
HAL_PCDEx_PMAConfig     0x08003129    0x36  Code  Gb  stm32l0xx_hal_pcd_ex.o [1]
HAL_PCD_DataInStageCallback
                        0x08002a0b    0x16  Code  Gb  usbd_conf.o [1]
HAL_PCD_DataOutStageCallback
                        0x080029f3    0x18  Code  Gb  usbd_conf.o [1]
HAL_PCD_DeInit          0x08001d25    0x26  Code  Gb  stm32l0xx_hal_pcd.o [1]
HAL_PCD_EP_Close        0x08002151   0x156  Code  Gb  stm32l0xx_hal_pcd.o [1]
HAL_PCD_EP_ClrStall     0x08002549    0x9a  Code  Gb  stm32l0xx_hal_pcd.o [1]
HAL_PCD_EP_Open         0x08001e95   0x294  Code  Gb  stm32l0xx_hal_pcd.o [1]
HAL_PCD_EP_Receive      0x080022b3    0xd0  Code  Gb  stm32l0xx_hal_pcd.o [1]
HAL_PCD_EP_SetStall     0x080024c9    0x7a  Code  Gb  stm32l0xx_hal_pcd.o [1]
HAL_PCD_EP_Transmit     0x0800239d   0x12c  Code  Gb  stm32l0xx_hal_pcd.o [1]
HAL_PCD_IRQHandler      0x08001d87    0xc2  Code  Gb  stm32l0xx_hal_pcd.o [1]
HAL_PCD_Init            0x08001c99    0x8c  Code  Gb  stm32l0xx_hal_pcd.o [1]
HAL_PCD_MspDeInit       0x080029a7    0x38  Code  Gb  usbd_conf.o [1]
HAL_PCD_MspInit         0x0800295d    0x4a  Code  Gb  usbd_conf.o [1]
HAL_PCD_ResetCallback   0x08002a2f    0x18  Code  Gb  usbd_conf.o [1]
HAL_PCD_ResumeCallback  0x08002a49     0x2  Code  Gb  usbd_conf.o [1]
HAL_PCD_SOFCallback     0x08002a21     0xe  Code  Gb  usbd_conf.o [1]
HAL_PCD_SetAddress      0x08001e69    0x2c  Code  Gb  stm32l0xx_hal_pcd.o [1]
HAL_PCD_SetupStageCallback
                        0x080029df    0x14  Code  Gb  usbd_conf.o [1]
HAL_PCD_Start           0x08001d4b    0x14  Code  Gb  stm32l0xx_hal_pcd.o [1]
HAL_PCD_Stop            0x08001d5f    0x28  Code  Gb  stm32l0xx_hal_pcd.o [1]
HAL_PCD_SuspendCallback
                        0x08002a47     0x2  Code  Gb  usbd_conf.o [1]
HAL_PWREx_EnableFastWakeUp
                        0x080066e5     0xc  Code  Gb  stm32l0xx_hal_pwr_ex.o [1]
HAL_PWREx_EnableUltraLowPower
                        0x080066f1     0xc  Code  Gb  stm32l0xx_hal_pwr_ex.o [1]
HAL_PWR_EnterSLEEPMode  0x080066b5    0x28  Code  Gb  stm32l0xx_hal_pwr.o [1]
HAL_RCCEx_CRSConfig     0x080054db    0x74  Code  Gb  stm32l0xx_hal_rcc_ex.o [1]
HAL_RCCEx_PeriphCLKConfig
                        0x080053b9   0x122  Code  Gb  stm32l0xx_hal_rcc_ex.o [1]
HAL_RCC_ClockConfig     0x08005105   0x1ec  Code  Gb  stm32l0xx_hal_rcc.o [1]
HAL_RCC_GetHCLKFreq     0x08005365    0x1a  Code  Gb  stm32l0xx_hal_rcc.o [1]
HAL_RCC_GetSysClockFreq
                        0x080052f9    0x60  Code  Gb  stm32l0xx_hal_rcc.o [1]
HAL_RCC_OscConfig       0x08004d4d   0x39a  Code  Gb  stm32l0xx_hal_rcc.o [1]
HAL_ResumeTick          0x080040f3     0x4  Code  Wk  stm32l0xx_hal.o [1]
HAL_SPI_DeInit          0x08005e63    0x30  Code  Gb  stm32l0xx_hal_spi.o [1]
HAL_SPI_GetState        0x08005ff1     0x6  Code  Gb  stm32l0xx_hal_spi.o [1]
HAL_SPI_Init            0x08005de1    0x82  Code  Gb  stm32l0xx_hal_spi.o [1]
HAL_SPI_MspDeInit       0x08005e95     0x2  Code  Wk  stm32l0xx_hal_spi.o [1]
HAL_SPI_MspInit         0x08005e93     0x2  Code  Wk  stm32l0xx_hal_spi.o [1]
HAL_SPI_Transmit        0x08005e97   0x150  Code  Gb  stm32l0xx_hal_spi.o [1]
HAL_SYSTICK_Config      0x08002e7f    0x28  Code  Gb  stm32l0xx_hal_cortex.o [1]
HAL_SuspendTick         0x080040ef     0x4  Code  Wk  stm32l0xx_hal.o [1]
HAL_TSC_DeInit          0x08004d0d    0x1e  Code  Gb  stm32l0xx_hal_tsc.o [1]
HAL_TSC_Init            0x08004c71    0x9c  Code  Gb  stm32l0xx_hal_tsc.o [1]
HAL_TSC_MspDeInit       0x080055fd    0x5c  Code  Gb  stm32l0xx_hal_msp.o [1]
HAL_TSC_MspInit         0x08005593    0x6a  Code  Gb  stm32l0xx_hal_msp.o [1]
HID_Buffer              0x2000108c     0x4  Data  Gb  usbdapp.o [1]
HID_Desc                0x2000096c    0x1c  Data  Gb  usbd_desc.o [1]
HID_MOUSE_ReportDesc    0x20000868    0x4c  Data  Lc  usbd_hid.o [1]
HardFault_Handler       0x08007f2b     0x2  Code  Gb  stm32l0xx_it.o [1]
I2C_Config              0x08004c19    0x36  Code  Lc  power.o [1]
I2C_IsAcknowledgeFailed
                        0x080065bb    0x88  Code  Lc  stm32l0xx_hal_i2c.o [1]
I2C_RequestMemoryRead   0x08006439    0x6c  Code  Lc  stm32l0xx_hal_i2c.o [1]
I2C_RequestMemoryWrite  0x080063cd    0x6c  Code  Lc  stm32l0xx_hal_i2c.o [1]
I2C_TransferConfig      0x08006655    0x1e  Code  Lc  stm32l0xx_hal_i2c.o [1]
I2C_WaitOnFlagUntilTimeout
                        0x080064a5    0x78  Code  Lc  stm32l0xx_hal_i2c.o [1]
I2C_WaitOnSTOPFlagUntilTimeout
                        0x08006577    0x44  Code  Lc  stm32l0xx_hal_i2c.o [1]
I2C_WaitOnTXISFlagUntilTimeout
                        0x0800651d    0x5a  Code  Lc  stm32l0xx_hal_i2c.o [1]
I2CxHandle              0x20000ebc    0x38  Data  Gb  power.o [1]
IDD_RestoreContext      0x0800373b    0xc2  Code  Gb  menu.o [1]
IDD_SaveContext         0x08003611   0x12a  Code  Gb  menu.o [1]
Idd_LPSleep_process     0x08004961   0x29a  Code  Gb  power.o [1]
Idd_Run_process         0x0800458d   0x1a4  Code  Gb  power.o [1]
Idd_Sleep_process       0x08004739   0x202  Code  Gb  power.o [1]
Idd_measurement         0x20000ef4     0x4  Data  Gb  power.o [1]
InStream_Read           0x08007b41    0x22  Code  Lc  lz77_init.o [4]
IntToUnicode            0x08007ea1    0x26  Code  Lc  usbd_desc.o [1]
LoadInt                 0x08006ab1    0x4c  Code  Lc  xprintfsmall_nomb.o [3]
MSIRangeTable           0x0800539c    0x1c  Data  Gb  stm32l0xx_hal_rcc.o [1]
Menu_Process            0x08003169   0x320  Code  Gb  menu.o [1]
MyBanks                 0x080041b4    0x18  Data  Gb  tsl_user.o [1]
MyChannels_Data         0x20001008    0x24  Data  Gb  tsl_user.o [1]
MyChannels_Dest         0x08007d38     0x8  Data  Gb  tsl_user.o [1]
MyChannels_Src          0x08007d14    0x24  Data  Gb  tsl_user.o [1]
MyLinRot0_DeltaCoeff    0x08007dec     0x8  Data  Gb  tsl_user.o [1]
MyLinRots               0x08007df4    0x24  Data  Gb  tsl_user.o [1]
MyLinRots_Data          0x2000107c     0x8  Data  Gb  tsl_user.o [1]
MyLinRots_ErrorStateProcess
                        0x080041ad     0x2  Code  Gb  tsl_user.o [1]
MyLinRots_Methods       0x08007de0     0xc  Data  Gb  tsl_user.o [1]
MyLinRots_OffStateProcess
                        0x080041af     0x2  Code  Gb  tsl_user.o [1]
MyLinRots_Param         0x2000105c    0x10  Data  Gb  tsl_user.o [1]
MyLinRots_StateMachine  0x08007d40    0xa0  Data  Gb  tsl_user.o [1]
MyObjGroup              0x2000095c    0x10  Data  Gb  tsl_user.o [1]
MyObjects               0x08007e18     0x8  Data  Gb  tsl_user.o [1]
NMI_Handler             0x08007f29     0x2  Code  Gb  stm32l0xx_it.o [1]
NVIC_SetPriority        0x08002e29    0x32  Code  Lc  stm32l0xx_hal_cortex.o [1]
OutStream_Write         0x08007b63    0x42  Code  Lc  lz77_init.o [4]
PCD_EP_ISR_Handler      0x08002605   0x2f0  Code  Lc  stm32l0xx_hal_pcd.o [1]
PCD_ReadPMA             0x08002941    0x1c  Code  Gb  stm32l0xx_hal_pcd.o [1]
PCD_WritePMA            0x0800291d    0x24  Code  Gb  stm32l0xx_hal_pcd.o [1]
PLLMulTable             0x200009dc     0xc  Data  Lc  stm32l0xx_hal_rcc.o [1]
PLLMulTable             0x20000940     0xc  Data  Gb  system_stm32l0xx.o [1]
PendSV_Handler          0x08007f31     0x2  Code  Gb  stm32l0xx_it.o [1]
Region$$Table$$Base     0x0800805c           --   Gb  - Linker created -
Region$$Table$$Limit    0x08008088           --   Gb  - Linker created -
RunModeMeasure          0x20000ef8     0x4  Data  Gb  power.o [1]
SPI_WaitOnFlagUntilTimeout
                        0x08005ff7    0xc2  Code  Lc  stm32l0xx_hal_spi.o [1]
SPIx_Error              0x08004449     0xe  Code  Lc  stm32l0538_discovery.o [1]
SPIx_Init               0x080043b5    0x7a  Code  Lc  stm32l0538_discovery.o [1]
SPIx_Write              0x0800442f    0x1a  Code  Lc  stm32l0538_discovery.o [1]
SVC_Handler             0x08007f2d     0x2  Code  Gb  stm32l0xx_it.o [1]
SoftDelay               0x080058cd     0xc  Code  Lc  tsl_acq_tsc.o [1]
SpiHandle               0x20000f74    0x54  Data  Lc  stm32l0538_discovery.o [1]
SysTick_Handler         0x08007f33    0x2c  Code  Gb  stm32l0xx_it.o [1]
SystemClock_Config      0x080037fd    0x4e  Code  Gb  menu.o [1]
SystemCoreClock         0x2000094c     0x4  Data  Gb  system_stm32l0xx.o [1]
SystemInit              0x08007f8d    0x40  Code  Gb  system_stm32l0xx.o [1]
TSC_extract_groups      0x08004d2b    0x22  Code  Lc  stm32l0xx_hal_tsc.o [1]
TSL_Globals             0x20001044    0x18  Data  Gb  tsl_globals.o [1]
TSL_Init                0x080057c1    0x30  Code  Gb  tsl.o [1]
TSL_POSOFF_3CH_LIN_H    0x080080d0    0x14  Data  Gb  tsl_linrot.o [1]
TSL_Params              0x200009cc    0x10  Data  Gb  tsl_user.o [1]
TSL_acq_BankConfig      0x080057f1    0x58  Code  Gb  tsl_acq_tsc.o [1]
TSL_acq_BankGetResult   0x080058d9   0x144  Code  Gb  tsl_acq.o [1]
TSL_acq_BankStartAcq    0x08005849    0x26  Code  Gb  tsl_acq_tsc.o [1]
TSL_acq_BankWaitEOC     0x0800586f    0x20  Code  Gb  tsl_acq_tsc.o [1]
TSL_acq_CheckNoise      0x080058bd     0x4  Code  Gb  tsl_acq_tsc.o [1]
TSL_acq_ComputeDelta    0x080058b1     0x6  Code  Gb  tsl_acq_tsc.o [1]
TSL_acq_ComputeMeas     0x080058b7     0x6  Code  Gb  tsl_acq_tsc.o [1]
TSL_acq_GetMeas         0x0800588f    0x12  Code  Gb  tsl_acq_tsc.o [1]
TSL_acq_TestFirstReferenceIsValid
                        0x080058c9     0x4  Code  Gb  tsl_acq_tsc.o [1]
TSL_acq_TestReferenceOutOfRange
                        0x080058c5     0x4  Code  Gb  tsl_acq_tsc.o [1]
TSL_acq_UseFilter       0x080058c1     0x4  Code  Gb  tsl_acq_tsc.o [1]
TSL_dxs_FirstObj        0x08005a25     0x2  Code  Gb  tsl_dxs.o [1]
TSL_ecs_CalcK           0x08005ab1    0xb2  Code  Gb  tsl_ecs.o [1]
TSL_ecs_Process         0x08005c21    0x72  Code  Gb  tsl_ecs.o [1]
TSL_ecs_ProcessK        0x08005b63    0xbe  Code  Gb  tsl_ecs.o [1]
TSL_linrot_CalcPos      0x08006d21   0x27e  Code  Gb  tsl_linrot.o [1]
TSL_linrot_CalibrationStateProcess
                        0x080071c9    0xba  Code  Gb  tsl_linrot.o [1]
TSL_linrot_DTOGetTime   0x080076eb    0x2c  Code  Gb  tsl_linrot.o [1]
TSL_linrot_DebCalibrationStateProcess
                        0x0800717b    0x42  Code  Gb  tsl_linrot.o [1]
TSL_linrot_DebDetectStateProcess
                        0x0800747d    0x6a  Code  Gb  tsl_linrot.o [1]
TSL_linrot_DebErrorStateProcess
                        0x08007679    0x72  Code  Gb  tsl_linrot.o [1]
TSL_linrot_DebProxDetectStateProcess
                        0x080072f5    0x6c  Code  Gb  tsl_linrot.o [1]
TSL_linrot_DebProxStateProcess
                        0x08007283    0x6a  Code  Gb  tsl_linrot.o [1]
TSL_linrot_DebProxTouchStateProcess
                        0x08007361    0x6c  Code  Gb  tsl_linrot.o [1]
TSL_linrot_DebReleaseDetectStateProcess
                        0x08007037    0x3a  Code  Gb  tsl_linrot.o [1]
TSL_linrot_DebReleaseProxStateProcess
                        0x0800700f    0x28  Code  Gb  tsl_linrot.o [1]
TSL_linrot_DebReleaseTouchStateProcess
                        0x0800708d    0x3c  Code  Gb  tsl_linrot.o [1]
TSL_linrot_DetectStateProcess
                        0x080074f1    0xc2  Code  Gb  tsl_linrot.o [1]
TSL_linrot_GetStateMask
                        0x08006ff1    0x1e  Code  Gb  tsl_linrot.o [1]
TSL_linrot_Init         0x08006c61    0x6a  Code  Gb  tsl_linrot.o [1]
TSL_linrot_Process      0x08006ccb    0x50  Code  Gb  tsl_linrot.o [1]
TSL_linrot_ProcessCh_All_ClearRef
                        0x0800783d    0x22  Code  Gb  tsl_linrot.o [1]
TSL_linrot_ProcessCh_All_DeltaBelowEqu
                        0x08007815    0x28  Code  Gb  tsl_linrot.o [1]
TSL_linrot_ProcessCh_All_SetStatus
                        0x08007717    0x2a  Code  Gb  tsl_linrot.o [1]
TSL_linrot_ProcessCh_One_AcqStatusError
                        0x0800776b    0x28  Code  Gb  tsl_linrot.o [1]
TSL_linrot_ProcessCh_One_DataReady
                        0x08007741    0x2a  Code  Gb  tsl_linrot.o [1]
TSL_linrot_ProcessCh_One_DeltaAbove
                        0x080077ed    0x28  Code  Gb  tsl_linrot.o [1]
TSL_linrot_ProcessCh_One_DeltaAboveEqu
                        0x080077bd    0x28  Code  Gb  tsl_linrot.o [1]
TSL_linrot_ProcessCh_One_DeltaBelowEquMinus
                        0x08007793    0x2a  Code  Gb  tsl_linrot.o [1]
TSL_linrot_ProxStateProcess
                        0x080073d7    0xa2  Code  Gb  tsl_linrot.o [1]
TSL_linrot_ReleaseStateProcess
                        0x080070d5    0xa6  Code  Gb  tsl_linrot.o [1]
TSL_linrot_SetStateCalibration
                        0x08006f9f    0x4c  Code  Gb  tsl_linrot.o [1]
TSL_linrot_TouchStateProcess
                        0x080075b3    0xc2  Code  Gb  tsl_linrot.o [1]
TSL_obj_GroupInit       0x08005701    0x54  Code  Gb  tsl_object.o [1]
TSL_obj_GroupProcess    0x08005755    0x54  Code  Gb  tsl_object.o [1]
TSL_obj_SetGlobalObj    0x080057a9    0x12  Code  Gb  tsl_object.o [1]
TSL_tim_CheckDelay_ms   0x08005a29    0x2a  Code  Gb  tsl_time.o [1]
TSL_tim_CheckDelay_sec  0x08005a53    0x34  Code  Gb  tsl_time.o [1]
TscHandle               0x20000fc8    0x40  Data  Gb  bsp.o [1]
USBClock_Disable        0x08003891    0x20  Code  Gb  menu.o [1]
USBClock_Enable         0x0800384b    0x46  Code  Gb  menu.o [1]
USBD_ClrClassConfig     0x08002f57     0xa  Code  Gb  usbd_core.o [1]
USBD_CtlContinueRx      0x08003d01     0x8  Code  Gb  usbd_ioreq.o [1]
USBD_CtlContinueSendData
                        0x08003cf9     0x8  Code  Gb  usbd_ioreq.o [1]
USBD_CtlError           0x08003c81    0x14  Code  Gb  usbd_ctlreq.o [1]
USBD_CtlReceiveStatus   0x08003d21     0xe  Code  Gb  usbd_ioreq.o [1]
USBD_CtlSendData        0x08003cd9    0x20  Code  Gb  usbd_ioreq.o [1]
USBD_CtlSendStatus      0x08003d09     0xe  Code  Gb  usbd_ioreq.o [1]
USBD_DeInit             0x08002ef3    0x2a  Code  Gb  usbd_core.o [1]
USBD_Device             0x20000a08   0x224  Data  Gb  bsp.o [1]
USBD_DeviceDesc         0x08007f10    0x14  Data  Gb  usbd_desc.o [1]
USBD_GetDescriptor      0x08003b5d    0xfc  Code  Lc  usbd_ctlreq.o [1]
USBD_GetString          0x08003c95    0x44  Code  Gb  usbd_ctlreq.o [1]
USBD_HID                0x200008b4    0x38  Data  Gb  usbd_hid.o [1]
USBD_HID_CfgDesc        0x200008ec    0x24  Data  Lc  usbd_hid.o [1]
USBD_HID_ConfigStrDescriptor
                        0x08007e7d     0xc  Code  Gb  usbd_desc.o [1]
USBD_HID_DataIn         0x08005dbf     0xe  Code  Lc  usbd_hid.o [1]
USBD_HID_DeInit         0x08005ccd    0x22  Code  Lc  usbd_hid.o [1]
USBD_HID_Desc           0x2000085c     0xc  Data  Lc  usbd_hid.o [1]
USBD_HID_DeviceDescriptor
                        0x08007e21     0x8  Code  Gb  usbd_desc.o [1]
USBD_HID_DeviceQualifierDesc
                        0x200009e8     0xc  Data  Lc  usbd_hid.o [1]
USBD_HID_GetCfgDesc     0x08005db7     0x8  Code  Lc  usbd_hid.o [1]
USBD_HID_GetDeviceQualifierDesc
                        0x08005dcd     0x8  Code  Lc  usbd_hid.o [1]
USBD_HID_Init           0x08005ca1    0x2c  Code  Lc  usbd_hid.o [1]
USBD_HID_InterfaceStrDescriptor
                        0x08007e89     0xc  Code  Gb  usbd_desc.o [1]
USBD_HID_LangIDStrDescriptor
                        0x08007e29     0x8  Code  Gb  usbd_desc.o [1]
USBD_HID_ManufacturerStrDescriptor
                        0x08007e3d     0xa  Code  Gb  usbd_desc.o [1]
USBD_HID_ProductStrDescriptor
                        0x08007e31     0xc  Code  Gb  usbd_desc.o [1]
USBD_HID_SendReport     0x08005d8f    0x28  Code  Gb  usbd_hid.o [1]
USBD_HID_SerialStrDescriptor
                        0x08007e4f    0x2c  Code  Gb  usbd_desc.o [1]
USBD_HID_Setup          0x08005cef    0xa0  Code  Lc  usbd_hid.o [1]
USBD_Init               0x08002ebd    0x36  Code  Gb  usbd_core.o [1]
USBD_LL_ClearStallEP    0x08002b03    0x10  Code  Gb  usbd_conf.o [1]
USBD_LL_CloseEP         0x08002ae3    0x10  Code  Gb  usbd_conf.o [1]
USBD_LL_DataInStage     0x08003025    0x94  Code  Gb  usbd_core.o [1]
USBD_LL_DataOutStage    0x08002fbb    0x6a  Code  Gb  usbd_core.o [1]
USBD_LL_DeInit          0x08002a9d    0x10  Code  Gb  usbd_conf.o [1]
USBD_LL_Init            0x08002a4b    0x52  Code  Gb  usbd_conf.o [1]
USBD_LL_IsStallEP       0x08002b13    0x1e  Code  Gb  usbd_conf.o [1]
USBD_LL_OpenEP          0x08002acd    0x16  Code  Gb  usbd_conf.o [1]
USBD_LL_PrepareReceive  0x08002b51    0x10  Code  Gb  usbd_conf.o [1]
USBD_LL_Reset           0x080030b9    0x46  Code  Gb  usbd_core.o [1]
USBD_LL_SOF             0x08003105    0x1c  Code  Gb  usbd_core.o [1]
USBD_LL_SetSpeed        0x080030ff     0x6  Code  Gb  usbd_core.o [1]
USBD_LL_SetUSBAddress   0x08002b31    0x10  Code  Gb  usbd_conf.o [1]
USBD_LL_SetupStage      0x08002f61    0x5a  Code  Gb  usbd_core.o [1]
USBD_LL_StallEP         0x08002af3    0x10  Code  Gb  usbd_conf.o [1]
USBD_LL_Start           0x08002aad    0x10  Code  Gb  usbd_conf.o [1]
USBD_LL_Stop            0x08002abd    0x10  Code  Gb  usbd_conf.o [1]
USBD_LL_Transmit        0x08002b41    0x10  Code  Gb  usbd_conf.o [1]
USBD_LangIDDesc         0x08007f24     0x4  Data  Gb  usbd_desc.o [1]
USBD_ParseSetupRequest  0x08003c59    0x28  Code  Gb  usbd_ctlreq.o [1]
USBD_RegisterClass      0x08002f1d    0x14  Code  Gb  usbd_core.o [1]
USBD_SetClassConfig     0x08002f3b    0x1c  Code  Gb  usbd_core.o [1]
USBD_Start              0x08002f31     0xa  Code  Gb  usbd_core.o [1]
USBD_StdDevReq          0x08003909   0x14c  Code  Gb  usbd_ctlreq.o [1]
USBD_StdEPReq           0x08003a93    0xca  Code  Gb  usbd_ctlreq.o [1]
USBD_StdItfReq          0x08003a59    0x3a  Code  Gb  usbd_ctlreq.o [1]
USBD_StrDesc            0x20000da4   0x100  Data  Gb  usbd_desc.o [1]
USBD_StringSerial       0x20000988    0x1c  Data  Gb  usbd_desc.o [1]
USBD_static_free        0x08002b81     0x2  Code  Gb  usbd_conf.o [1]
USBD_static_malloc      0x08002b61     0x4  Code  Gb  usbd_conf.o [1]
USB_IRQHandler          0x08007f5f     0xa  Code  Gb  stm32l0xx_it.o [1]
USB_process             0x08004297    0x30  Code  Gb  usbdapp.o [1]
WF_LUT                  0x08007ae4    0x5c  Data  Gb  gde021a1.o [1]
_LitobSmallNoMb         0x08006afd    0xf2  Code  Lc  xprintfsmall_nomb.o [3]
_PrintfSmallNoMb        0x08006701   0x3a4  Code  Gb  xprintfsmall_nomb.o [3]
_PutcharsSmallNoMb      0x08006bf5    0x30  Code  Lc  xprintfsmall_nomb.o [3]
_SProut                 0x0800315f     0xa  Code  Gb  xsprout.o [3]
__aeabi_idiv            0x08003d65          Code  Gb  I32DivModFast.o [4]
__aeabi_idiv0           0x0800558d          Code  Gb  IntDivZer.o [4]
__aeabi_idivmod         0x08003d65          Code  Gb  I32DivModFast.o [4]
__aeabi_uidiv           0x08003d6b          Code  Gb  I32DivModFast.o [4]
__aeabi_uidivmod        0x08003d6b          Code  Gb  I32DivModFast.o [4]
__as_entries_start      0xffffffff           --   Gb  command line/config [2]
__as_table_start        0xffffffff           --   Gb  command line/config [2]
__cmain                 0x08008089          Code  Gb  cmain.o [4]
__exit                  0x08007d09          Code  Gb  XXexit.o [4]
__iar_Memchr            0x08006c49    0x18  Code  Gb  memchr.o [4]
__iar_Strchr            0x08006c25    0x14  Code  Gb  strchr.o [4]
__iar_data_init3        0x08008035    0x28  Code  Gb  data_init.o [4]
__iar_lz77_init3        0x08007ba5   0x15a  Code  Gb  lz77_init.o [4]
__iar_program_start     0x080080f5          Code  Gb  cstartup_M.o [4]
__iar_zero_init3        0x08002b83    0x2a  Code  Gb  zero_init3.o [4]
__low_level_init        0x080080a3     0x4  Code  Gb  low_level_init.o [3]
__vector_table          0x08000000          Data  Gb  startup_stm32l053xx.o [1]
_call_main              0x08008095          Code  Gb  cmain.o [4]
_exit                   0x080080c5          Code  Gb  cexit.o [4]
_main                   0x0800809f          Code  Gb  cmain.o [4]
aRxBuffer               0x20000eb8     0x4  Data  Gb  power.o [1]
abort                   0x08007cff     0xa  Code  Gb  abort.o [3]
epd_drv                 0x200009a8     0x4  Data  Lc  stm32l0538_discovery_epd.o [1]
exit                    0x080080bb     0x8  Code  Gb  exit.o [3]
gde021a1_CloseChargePump
                        0x0800797d     0xa  Code  Gb  gde021a1.o [1]
gde021a1_DrawImage      0x08007993   0x150  Code  Gb  gde021a1.o [1]
gde021a1_GetEpdPixelHeight
                        0x08007961     0x4  Code  Gb  gde021a1.o [1]
gde021a1_GetEpdPixelWidth
                        0x0800795d     0x4  Code  Gb  gde021a1.o [1]
gde021a1_Init           0x08007869    0xa4  Code  Gb  gde021a1.o [1]
gde021a1_RefreshDisplay
                        0x08007971     0xc  Code  Gb  gde021a1.o [1]
gde021a1_SetDisplayWindow
                        0x08007915    0x48  Code  Gb  gde021a1.o [1]
gde021a1_WritePixel     0x0800790d     0x8  Code  Gb  gde021a1.o [1]
gde021a1_drv            0x20000910    0x20  Data  Gb  gde021a1.o [1]
hpcd                    0x20000c2c   0x178  Data  Gb  usbd_conf.o [1]
main                    0x080080a7    0x14  Code  Gb  main.o [1]
menu_state              0x20000000     0x1  Data  Gb  menu.o [1]
pFont                   0x200009a4     0x4  Data  Lc  stm32l0538_discovery_epd.o [1]
param                   0x20000ea4    0x14  Data  Gb  power.o [1]
sprintf                 0x0800667d    0x38  Code  Gb  sprintf.o [3]
str                     0x20000efc    0x14  Data  Gb  power.o [1]
strlen                  0x08006c39    0x10  Code  Gb  strlen.o [4]
tsl_user_Exec           0x08004129    0x7c  Code  Gb  tsl_user.o [1]
tsl_user_Init           0x08004119    0x10  Code  Gb  tsl_user.o [1]
uwTick                  0x20001084     0x4  Data  Lc  stm32l0xx_hal.o [1]


[1] = C:\ESEMPI-SW\STM32L0\STM32Cube_FW_L0_V1.1.0\Projects\STM32L053C8-Discovery\Demonstrations\EWARM\STM32L0538-Discovery\Obj
[2] = command line
[3] = dl6M_tlf.a
[4] = rt6M_tl.a

  25 518 bytes of readonly  code memory
   8 325 bytes of readonly  data memory
   6 291 bytes of readwrite data memory

Errors: none
Warnings: none
